:020000040000FA
:04080000F2EF07F01C
:1008100003B213EF05F0F2B431EF05F09EB039EFFB
:1008200005F09EB241EF05F0F2A81AEF04F0F2B223
:1008300025EF04F0F2A620EF04F0F2B022EF04F06E
:10084000A1EF07F0F296F290FF00CD90F2929EA0F9
:100850002FEF04F00101533F2FEF04F0542BAEC1F2
:10086000B2F1AFC1B3F1B0C1B4F1B1C1B5F1AAC138
:10087000AEF1ABC1AFF1ACC1B0F1ADC1B1F1A6C148
:10088000AAF1A7C1ABF1A8C1ACF1A9C1ADF1A2C158
:10089000A6F1A3C1A7F1A4C1A8F1A5C1A9F19EC168
:1008A000A2F19FC1A3F1A0C1A4F1A1C1A5F19AC178
:1008B0009EF19BC19FF19CC1A0F19DC1A1F196C188
:1008C0009AF197C19BF198C19CF199C19DF1CECF4E
:1008D00096F1CFCF97F153C198F154C199F1CF6AF6
:1008E000CE6A0101536B546B9E90CD800FBC0F8E6E
:1008F0000FBA7EEF04F00F8AA1EF07F00F8C0FBE46
:10090000BAEF04F096C19AF197C19BF198C19CF19E
:1009100099C19DF19AC19EF19BC19FF19CC1A0F12B
:100920009DC1A1F19EC1A2F19FC1A3F1A0C1A4F1FB
:10093000A1C1A5F1A2C1A6F1A3C1A7F1A4C1A8F1CB
:10094000A5C1A9F1A6C1AAF1A7C1ABF1A8C1ACF19B
:10095000A9C1ADF1AAC1AEF1ABC1AFF1ACC1B0F16B
:10096000ADC1B1F1AEC1B2F1AFC1B3F1B0C1B4F13B
:10097000B1C1B5F101015E6B5F6B606B616B96514C
:100980005E2797515F2398516023995161239A51B3
:100990005E279B515F239C5160239D5161239E5193
:1009A0005E279F515F23A0516023A1516123A25173
:1009B0005E27A3515F23A4516023A5516123A65153
:1009C0005E27A7515F23A8516023A9516123AA5133
:1009D0005E27AB515F23AC516023AD516123AE5113
:1009E0005E27AF515F23B0516023B1516123B251F3
:1009F0005E27B3515F23B4516023B5516123D89072
:100A00000101613360335F335E33D890010161339C
:100A100060335F335E33D8900101613360335F33FD
:100A20005E33A1EF07F00392ABB2AB98AB88030142
:100A300003EE00F080517F0BE92604C0EFFF802B0E
:100A40008151805D700BD8A48B8200008051815D44
:100A5000700BD8A48B9281518019D8B40790A1EF64
:100A600007F0F2940101453FA1EF07F0462BA1EFFB
:100A700007F09E900101533FA1EF07F0542BA1EF27
:100A800007F09E92040062A146EF05F0077C07ACD8
:100A900061EF05F0C274C2B45BEF05F0C3CFB3F5EC
:100AA000C4CFB4F50501D890B433B333D890B43380
:100AB000B33362EF05F0C3CF55F1C4CF56F162EF07
:100AC00005F0C28207B4CFEF05F047C14BF148C132
:100AD0004CF149C14DF14AC14EF15EC162F15FC1B5
:100AE00063F160C164F161C165F196C1B6F197C16E
:100AF000B7F198C1B8F199C1B9F19AC1BAF19BC1E6
:100B0000BBF19CC1BCF19DC1BDF19EC1BEF19FC1B5
:100B1000BFF1A0C1C0F1A1C1C1F1A2C1C2F1A3C185
:100B2000C3F1A4C1C4F1A5C1C5F1A6C1C6F1A7C155
:100B3000C7F1A8C1C8F1A9C1C9F1AAC1CAF1ABC125
:100B4000CBF1ACC1CCF1ADC1CDF1AEC1CEF1AFC1F5
:100B5000CFF1B0C1D0F1B1C1D1F1B2C1D2F1B3C1C5
:100B6000D3F1B4C1D4F1B5C1D5F1B3C5B5F5B4C5B0
:100B7000B6F5B5C5B7F5B6C5B8F5010155515B2752
:100B800056515C23E86A5D230E2ECFEF05F05CC161
:100B900057F15DC158F15B6B5C6B5D6B078E0201B9
:100BA000002FA1EF07F03C0E006F00C10CF101C156
:100BB0000DF102C10EF103C10FF104C110F105C125
:100BC00011F106C112F107C113F108C114F109C1F5
:100BD00015F10AC116F10BC117F134C135F1050148
:100BE0002F51000AD8B4A0EF06F005012F51010AD9
:100BF000D8B42AEF06F005012F51020AD8B46BEFE2
:100C000006F005012F51030AD8B46BEF06F0050179
:100C10002F51040AD8B46BEF06F005012F51050AD5
:100C2000D8B46BEF06F005012F51060AD8B46BEF6C
:100C300006F005012F51070AD8B46BEF06F0050145
:100C40002F51320AD8B428EF06F02F6BA0EF06F030
:100C5000A0EF06F00501536735EF06F0546735EF56
:100C600006F0556735EF06F0566739EF06F0A0EF4E
:100C700006F057C500F158C501F159C502F15AC532
:100C800003F10101010E046F000E056F000E066FE7
:100C9000000E076F08EC20F000C157F501C158F5B0
:100CA00002C159F503C15AF500675EEF06F001670E
:100CB0005EEF06F002675EEF06F00367A0EF06F056
:100CC00053C557F554C558F555C559F556C55AF588
:100CD0000F88A0EF06F00501306771EF06F0A0EF76
:100CE00006F00FBE86EF06F010A08BEF06F00101B4
:100CF000476782EF06F0486782EF06F0496782EFA8
:100D000006F04A6786EF06F08BEF06F007AE8BEF32
:100D100006F09DEF06F00501312FA0EF06F03C0E26
:100D2000316F302FA0EF06F00101000E626FE00E70
:100D3000636FA50E646F010E656F0501306B0F8840
:100D40000501626B33B7A6EF06F062810CC100F1BA
:100D50000DC101F10EC102F10FC103F110C104F187
:100D600011C105F112C106F113C107F114C108F157
:100D700015C109F116C10AF117C10BF135C134F1E2
:100D800000C10CF101C10DF102C10EF103C10FF15F
:100D900004C110F105C111F106C112F107C113F12F
:100DA00008C114F109C115F10AC116F10BC117F1FF
:100DB00034C135F101018A67E5EF06F08B67E5EF95
:100DC00006F08C67E5EF06F08D67E9EF06F019EFA6
:100DD00007F08EC100F18FC101F190C102F191C104
:100DE00003F10101010E046F000E056F000E066F86
:100DF000000E076F08EC20F000C18EF101C18FF1E9
:100E000002C190F103C191F100670EEF07F0016795
:100E10000EEF07F002670EEF07F0036719EF07F018
:100E20008AC18EF18BC18FF18CC190F18DC191F18E
:100E30000F80D57ED5BE69D0D6CF47F1D7CF48F148
:100E400045C149F1E86AE8CF4AF1109047C100F185
:100E500048C101F149C102F14AC103F101010A0E81
:100E6000046F000E056F000E066F000E076F08EC92
:100E700020F003AF1080010154A74BEF07F00F9A49
:100E80000F9C0F9E0101000E5E6F600E5F6F3D0EA6
:100E9000606F080E616F010147BF5BEF07F04867A5
:100EA0005BEF07F049675BEF07F04A675BEF07F01E
:100EB000F28880EF07F0F2985E6B5F6B606B616B9E
:100EC000966B976B986B996B9A6B9B6B9C6B9D6BFE
:100ED0009E6B9F6BA06BA16BA26BA36BA46BA56BAE
:100EE000A66BA76BA86BA96BAA6BAB6BAC6BAD6B5E
:100EF000AE6BAF6BB06BB16BB26BB36BB46BB56B0E
:100F0000D76AD66A0101456B466B0CC100F10DC171
:100F100001F10EC102F10FC103F110C104F111C1C1
:100F200005F112C106F113C107F114C108F115C191
:100F300009F116C10AF117C10BF135C134F1A1EF66
:100F400007F002C0E0FF005001C0D8FF1000A6B2B9
:100F5000A7EF07F00CC0A9FF0BC0A8FFA69EA69C98
:100F6000A684F29E550EA76EAA0EA76EA682F28EDA
:100F7000A694A6B2B9EF07F00C2A1200A96EA69E9D
:100F8000A69CA680A8500C2A120004012C0E826F89
:100F9000CBEC0AF003EC21F00C50BEEC07F0E8CFEC
:100FA00000F10C50BEEC07F0E8CF01F101AFDEEF2D
:100FB00007F00101FF0E026FFF0E036FA6EC20F099
:100FC0002967EAEF07F00401200E826FCBEC0AF0EC
:100FD000EFEF07F004012D0E826FCBEC0AF0D0EC9E
:100FE0001EF01200076A0F6A106A0F010D0EC16E23
:100FF000860EC06E030EC26E0F01680E896E130E50
:10100000926E080E8A6EF30E936E8B6A900E946E3B
:10101000C80EBEEC07F0E8CFE8FF1098E8A01088F3
:1010200010A805D0150E0E6E160E8E6F04D0150E7C
:101030000F6E160E8F6F7BEC21F0F18EF19E0E6A13
:1010400001015B6B5C6B5D6B576B586BF29A010136
:10105000476B486B496B4A6B4B6B4C6B4D6B4E6BE4
:101060004F6B506B516B526B456B466BD76AD66AB0
:101070000F01280ED56EF28A9D90B00ECD6E010143
:101080005E6B5F6B606B616B626B636B646B656BFC
:10109000666B676B686B696B536B546BCF6ACE6A18
:1010A0000F9A0F9C0F9E9D80760ECA6E9D82020144
:1010B0003C0E006FCC6A160EBEEC07F0E8CF00F1D4
:1010C000170EBEEC07F0E8CF01F1180EBEEC07F0EA
:1010D000E8CF02F1190EBEEC07F0E8CF03F10101F1
:1010E00003AF8DEF08F003EC21F0160E0C6E00C17B
:1010F0000BF0A7EC07F0170E0C6E01C10BF0A7EC7C
:1011000007F0180E0C6E02C10BF0A7EC07F0190ED9
:101110000C6E03C10BF0A7EC07F000C18AF101C10E
:101120008BF102C18CF103C18DF100C18EF101C1BF
:101130008FF102C190F103C191F11A0EBEEC07F0DC
:10114000E8CF00F11B0EBEEC07F0E8CF01F11C0E5A
:10115000BEEC07F0E8CF02F11D0EBEEC07F0E8CFC1
:1011600003F1010103AFE3EF08F003EC21F01A0EE5
:101170000C6E00C10BF0A7EC07F01B0E0C6E01C14A
:101180000BF0A7EC07F01C0E0C6E02C10BF0A7ECE5
:1011900007F01D0E0C6E03C10BF0A7EC07F01A0E42
:1011A000BEEC07F0E8CF00F11B0EBEEC07F0E8CF75
:1011B00001F11C0EBEEC07F0E8CF02F11D0EBEECF3
:1011C00007F0E8CF03F100C192F101C193F102C130
:1011D00094F103C195F1240EAC6E900EAB6E240E0B
:1011E000AC6E080EB86E000EB06E1F0EAF6E04012E
:1011F000806B816B0F01900EAB6E0F019D8A030116
:10120000806B816BC26B8B9234EC26F034EC26F051
:1012100090EC27F013EC24F0200EBEEC07F0E8CFA2
:101220002FF505012F51FF0AD8A41EEF09F02F6BEF
:10123000200E0C6E2FC50BF0A7EC07F00501010E78
:10124000306F3C0E316F250EBEEC07F0E8CF00F199
:10125000260EBEEC07F0E8CF01F1270EBEEC07F03A
:10126000E8CF02F1280EBEEC07F0E8CF03F1010150
:1012700003AF55EF09F003EC21F0250E0C6E00C111
:101280000BF0A7EC07F0260E0C6E01C10BF0A7ECDB
:1012900007F0270E0C6E02C10BF0A7EC07F0280E2A
:1012A0000C6E03C10BF0A7EC07F000C153F501C1B0
:1012B00054F502C155F503C156F500C157F501C1FA
:1012C00058F502C159F503C15AF5290EBEEC07F0D5
:1012D000E8CF5BF505015C515B5DD8A05BC55CF5B3
:1012E00005012F51020A0EE181B882EF09F00501D4
:1012F0005C2F7FEF09F05BC55CF582EF09F081BAE6
:10130000CFEF27F0210EBEEC07F0E8CF00F1220E60
:10131000BEEC07F0E8CF01F1230EBEEC07F0E8CFFA
:1013200002F1240EBEEC07F0E8CF03F1010103AF98
:10133000C8EF09F003EC21F0210E0C6E00C10BF098
:10134000A7EC07F0220E0C6E01C10BF0A7EC07F022
:10135000230E0C6E02C10BF0A7EC07F0240E0C6EEE
:1013600003C10BF0A7EC07F0210EBEEC07F0E8CFAD
:1013700000F1220EBEEC07F0E8CF01F1230EBEEC27
:1013800007F0E8CF02F1240EBEEC07F0E8CF03F13E
:1013900000C15DF501C15EF502C15FF503C160F5F5
:1013A00037EC23F02DEC22F081EC21F005012F51D8
:1013B000030A12E005012F51040A1DE005012F5117
:1013C000050A24E005012F51060A32E005012F51DC
:1013D000070A38E02BEF0AF0ACC500F101010F0E4F
:1013E000001701010051000A36E001010051050A11
:1013F00032E028EF0AF0ACC500F101010F0E001732
:1014000001010051000A27E028EF0AF00501AC5164
:10141000000A21E00501AC51150A1DE00501AC519F
:10142000300A19E00501AC51450A15E028EF0AF031
:101430000501AC51000A0FE00501AC51300A0BE088
:1014400028EF0AF00501AC51000A05E028EF0AF088
:1014500081BACFEF27F007900001F28EF28C07B02F
:1014600051EF1DF00FB030EF18F00FB8F4EF11F09E
:101470000301805181197F0BD8B451EF1DF013EE99
:1014800000F081517F0BE126812BE7CFE8FFE00BD5
:10149000D8B451EF1DF023EE82F0C2513F0BD92694
:1014A000E7CFDFFFC22BDF50780AD8A451EF1DF041
:1014B00007808EC100F18FC101F190C102F191C18D
:1014C00003F10101040E046F000E056F000E066F9C
:1014D000000E076F08EC20F000AF78EF0AF0010172
:1014E000030E8E6F000E8F6F000E906F000E916FC7
:1014F00003018251720AD8B430EF18F08251520AB7
:10150000D8B430EF18F08251750AD8B430EF18F023
:101510008251630AD8B40BEF1AF08251690AD8B429
:10152000EBEF14F082517A0AD8B4FEEF15F0825135
:10153000490AD8B48AEF14F08251500AD8B4A8EFFF
:1015400013F08251700AD8B4EBEF13F08251540AB1
:10155000D8B416EF14F08251740AD8B45CEF14F0CA
:1015600082516D0AD8B4DFEF0AF082514D0AD8B427
:10157000F8EF0AF08251730AD8B460EF17F0825185
:10158000530AD8B4C5EF17F082514C0AD8B487EF8C
:101590000BF042EF1AF0040114EE00F080517F0BC3
:1015A000E12682C4E7FF802B120004010D0E826F3A
:1015B000CBEC0AF00A0E826FCBEC0AF012000401A9
:1015C0006D0E826FCBEC0AF003018351300AD8B460
:1015D00037EF0BF003018351310AD8B44AEF0BF017
:1015E00003018351320AD8B45DEF0BF042EF1AF0D9
:1015F00004014D0E826FCBEC0AF044EC21F084C361
:1016000031F185C332F186C333F10101296B51EC0D
:1016100021F0C8EC20F003018351300AD8B41FEF49
:101620000BF003018351310AD8B427EF0BF003010B
:101630008351320AD8B42FEF0BF042EF1AF0FD0EAF
:101640000C6E00C10BF0A7EC07F037EF0BF0FE0EAD
:101650000C6E00C10BF0A7EC07F04AEF0BF0FF0E89
:101660000C6E00C10BF0A7EC07F05DEF0BF004016E
:10167000300E826FCBEC0AF004012C0E826FCBECA3
:101680000AF003EC21F0FD0EBEEC07F0E8CF00F10C
:101690006EEF0BF00401310E826FCBEC0AF0040107
:1016A0002C0E826FCBEC0AF003EC21F0FE0EBEECA8
:1016B00007F0E8CF00F16EEF0BF00401320E826FFD
:1016C000CBEC0AF003EC21F004012C0E826FCBEC82
:1016D0000AF0FF0EBEEC07F0E8CF00F1A6EC20F018
:1016E00031C182F40401300E8227CBEC0AF032C102
:1016F00082F40401300E8227CBEC0AF033C182F46D
:101700000401300E8227CBEC0AF040EF1AF00301FF
:101710008351300AD8B4ECEF0EF003018351310A43
:10172000D8B4FAEF0FF003018351320AD8B468EF4E
:1017300010F003018351330AD8B478EF10F003019D
:101740008351340AD8B488EF10F003018351350A6D
:10175000D8B4F9EF11F003018351360AD8B427EF5A
:1017600012F003018351370AD8B44EEF0EF0030193
:101770008351460AD8B44DEF11F0030183514D0A4D
:10178000D8B4C7EF0CF0030183516D0AD8B4E1EF70
:101790000CF0030183515A0AD8B474EF0FF003011F
:1017A0008351490AD8B427EF13F003018351500A3B
:1017B000D8B459EF12F003018351540AD8B4D2EFD0
:1017C00012F003018351630AD8B401EF0DF0030155
:1017D0008351430AD8B4F9EF0DF003018351730A22
:1017E000D8B4FFEF0CF003018351610AD8B414EFB1
:1017F0000CF003018351650AD8B43CEF0FF00301EC
:101800008351450AD8B44AEF0FF003018351620AAD
:10181000D8B458EF0FF003018351420AD8B466EFF1
:101820000FF0D8A442EF1AF004014C0E826FCBECFB
:101830000AF00401610E826FCBEC0AF02DEC22F06D
:1018400004012C0E826FCBEC0AF003EC21F0ABC547
:1018500000F10101A6EC20F031C182F40401300E48
:101860008227CBEC0AF032C182F40401300E8227C9
:10187000CBEC0AF033C182F40401300E8227CBECAA
:101880000AF004012C0E826FCBEC0AF003EC21F07D
:10189000ACC500F10101A6EC20F031C182F40401D5
:1018A000300E8227CBEC0AF032C182F40401300EF4
:1018B0008227CBEC0AF033C182F40401300E822778
:1018C000CBEC0AF004012C0E826FCBEC0AF003EC97
:1018D00021F0ADC500F10101A6EC20F031C182F488
:1018E0000401300E8227CBEC0AF032C182F40401ED
:1018F000300E8227CBEC0AF033C182F40401300EA3
:101900008227CBEC0AF004012C0E826FCBEC0AF09C
:1019100003EC21F0AEC500F10101A6EC20F031C1CD
:1019200082F40401300E8227CBEC0AF032C182F43B
:101930000401300E8227CBEC0AF033C182F404019B
:10194000300E8227CBEC0AF004012C0E826FCBEC18
:101950000AF003EC21F0B2C500F10101A6EC20F081
:1019600031C182F40401300E8227CBEC0AF032C17F
:1019700082F40401300E8227CBEC0AF033C182F4EA
:101980000401300E8227CBEC0AF055EF12F044EC44
:1019900021F084C333F151EC21F0C8EC20F0200E8B
:1019A0000C6E00C10BF0A7EC07F000C12FF505018C
:1019B0002F51000A06E005012F51010A02E0CFEC89
:1019C00022F004014C0E826FCBEC0AF004014D0EA4
:1019D000826FCBEC0AF004012C0E826FCBEC0AF084
:1019E00003EC21F02FC500F1A6EC20F033C182F406
:1019F0000401300E8227CBEC0AF055EF12F0CFEF46
:101A000027F004014C0E826FCBEC0AF00401630E48
:101A1000826FCBEC0AF081EC21F004012C0E826F76
:101A2000CBEC0AF016EC0DF055EF12F003EC21F0C0
:101A3000B1C500F10101003B0F0E0017A6EC20F02C
:101A400033C182F40401300E8227CBEC0AF0B1C519
:101A500000F101010F0E01010017A6EC20F033C1C7
:101A600082F40401300E8227CBEC0AF004012D0E23
:101A7000826FCBEC0AF0B0C500F10101003B0F0E04
:101A80000017A6EC20F033C182F40401300E822747
:101A9000CBEC0AF0B0C500F101010F0E01010017F7
:101AA000A6EC20F033C182F40401300E8227CBEC87
:101AB0000AF004012D0E826FCBEC0AF0AFC500F1E5
:101AC0000101003B0F0E0017A6EC20F033C182F499
:101AD0000401300E8227CBEC0AF0AFC500F1010102
:101AE0000F0E01010017A6EC20F033C182F40401AF
:101AF000300E8227CBEC0AF00401200E826FCBEC73
:101B00000AF0AEC500F10F0E01010017A6EC20F09F
:101B100033C182F40401300E8227CBEC0AF00401B9
:101B2000200E826FCBEC0AF0ADC500F1010101017E
:101B3000003B0F0E0017A6EC20F033C182F4040125
:101B4000300E8227CBEC0AF0ADC500F101010F0E7B
:101B500001010017A6EC20F033C182F40401300E1D
:101B60008227CBEC0AF004013A0E826FCBEC0AF02C
:101B7000ACC500F10101003B0F0E0017A6EC20F0F0
:101B800033C182F40401300E8227CBEC0AF0ACC5DD
:101B900000F101010F0E01010017A6EC20F033C186
:101BA00082F40401300E8227CBEC0AF004013A0ED5
:101BB000826FCBEC0AF0ABC500F10101003B0F0EC8
:101BC0000017A6EC20F033C182F40401300E822706
:101BD000CBEC0AF0ABC500F101010F0E0017A6EC2B
:101BE00020F033C182F40401300E8227CBEC0AF0DE
:101BF000120084C3E8FF0F0BE83AE8CFB1F585C3C4
:101C0000E8FF0F0B0501B11387C3E8FF0F0BE83A9C
:101C1000E8CFB0F588C3E8FF0F0B0501B0138AC306
:101C2000E8FF0F0BE83AE8CFAFF58BC3E8FF0F0BE7
:101C30000501AF138DC3E8FF0F0BE8CFAEF58FC3DF
:101C4000E8FF0F0BE83AE8CFADF590C3E8FF0F0BC4
:101C50000501AD1392C3E8FF0F0BE83AE8CFACF5EE
:101C600093C3E8FF0F0B0501AC1395C3E8FF0F0BFF
:101C7000E83AE8CFABF596C3E8FF0F0B0501AB13CD
:101C8000DEEC21F004014C0E826FCBEC0AF0040173
:101C9000430E826FCBEC0AF00BEF0DF007840401CA
:101CA0004C0E826FCBEC0AF00401370E826FCBEC46
:101CB0000AF004012C0E826FCBEC0AF005012E51C4
:101CC000130A06E005012E51170A0DE0E9EF0EF0A8
:101CD0000101000E006F000E016F100E026F000E6A
:101CE000036F7CEF0EF00101000E006F000E016F1C
:101CF000000E026F010E036FA6EC20F02AC182F4E1
:101D00000401300E8227CBEC0AF02BC182F40401CF
:101D1000300E8227CBEC0AF02CC182F40401300E85
:101D20008227CBEC0AF02DC182F40401300E822709
:101D3000CBEC0AF02EC182F40401300E8227CBECEA
:101D40000AF02FC182F40401300E8227CBEC0AF096
:101D500030C182F40401300E8227CBEC0AF031C18D
:101D600082F40401300E8227CBEC0AF032C182F4F7
:101D70000401300E8227CBEC0AF033C182F4040157
:101D8000300E8227CBEC0AF004012C0E826FCBECD4
:101D90000AF00101100E006F000E016F000E026FBD
:101DA000000E036FA6EC20F031C182F40401300E66
:101DB0008227CBEC0AF032C182F40401300E822774
:101DC000CBEC0AF033C182F40401300E8227CBEC55
:101DD0000AF0079455EF12F0078490EC27F003EC1B
:101DE00021F02DC500F1A6EC20F004014C0E826F0D
:101DF000CBEC0AF00401300E826FCBEC0AF0040148
:101E00002C0E826FCBEC0AF031C182F40401300E4B
:101E10008227CBEC0AF032C182F40401300E822713
:101E2000CBEC0AF033C182F40401300E8227CBECF4
:101E30000AF004012C0E826FCBEC0AF003EC21F0C7
:101E40002EC500F1A6EC20F031C182F40401300E61
:101E50008227CBEC0AF032C182F40401300E8227D3
:101E6000CBEC0AF033C182F40401300E8227CBECB4
:101E70000AF0079455EF12F004014C0E826FCBEC80
:101E80000AF00401650E826FCBEC0AF0A3EC23F09C
:101E900055EF12F004014C0E826FCBEC0AF00401F6
:101EA000450E826FCBEC0AF0BEEC23F055EF12F03A
:101EB00004014C0E826FCBEC0AF00401620E826FBB
:101EC000CBEC0AF0F4EC23F055EF12F004014C0EC9
:101ED000826FCBEC0AF00401420E826FCBEC0AF069
:101EE000D9EC23F055EF12F004014C0E826FCBECCD
:101EF0000AF004015A0E826FCBEC0AF004012C0E9A
:101F0000826FCBEC0AF090EC27F003EC21F0050196
:101F10002E51130A06E005012E51170A0DE0A5EF18
:101F20000FF00101000E006F000E016F100E026F26
:101F3000000E036FA5EF0FF00101000E006F000E01
:101F4000016F000E026F010E036F0101100E046F8E
:101F5000000E056F000E066F000E076F39EC20F0C3
:101F6000A6EC20F02AC182F40401300E8227CBECCB
:101F70000AF02BC182F40401300E8227CBEC0AF068
:101F80002CC182F40401300E8227CBEC0AF02DC163
:101F900082F40401300E8227CBEC0AF02EC182F4C9
:101FA0000401300E8227CBEC0AF02FC182F4040129
:101FB000300E8227CBEC0AF030C182F40401300EDF
:101FC0008227CBEC0AF031C182F40401300E822763
:101FD000CBEC0AF032C182F40401300E8227CBEC44
:101FE0000AF033C182F40401300E8227CBEC0AF0F0
:101FF00055EF12F0078404014C0E826FCBEC0AF00F
:102000000401310E826FCBEC0AF004012C0E826FBA
:10201000CBEC0AF025C500F126C501F127C502F178
:1020200028C503F10101100E046F000E056F000EAC
:10203000066F000E076F39EC20F0A6EC20F02AC1E5
:1020400082F40401300E8227CBEC0AF02BC182F41B
:102050000401300E8227CBEC0AF02CC182F404017B
:10206000300E8227CBEC0AF02DC182F40401300E31
:102070008227CBEC0AF02EC182F40401300E8227B5
:10208000CBEC0AF02FC182F40401300E8227CBEC96
:102090000AF030C182F40401300E8227CBEC0AF042
:1020A00031C182F40401300E8227CBEC0AF032C138
:1020B00082F40401300E8227CBEC0AF033C182F4A3
:1020C0000401300E8227CBEC0AF0079455EF12F092
:1020D000078404014C0E826FCBEC0AF00401320E2F
:1020E000826FCBEC0AF0EAEC25F0079455EF12F082
:1020F000078404014C0E826FCBEC0AF00401330E0E
:10210000826FCBEC0AF047EC26F0079405EF10F055
:10211000078404014C0E826FCBEC0AF00401340EEC
:10212000826FCBEC0AF004012C0E826FCBEC0AF02C
:1021300044EC21F084C32AF185C32BF186C32CF132
:1021400087C32DF188C32EF189C32FF18AC330F1E3
:102150008BC331F18CC332F18DC333F10101296B93
:1021600051EC21F0C8EC20F0100E046F000E056F4A
:10217000000E066F000E076F19EC20F000C121F56C
:1021800001C122F502C123F503C124F543EC27F078
:1021900034C5ABF535C5ACF536C5ADF537C5AEF5CF
:1021A00038C5AFF539C5B0F53AC5B1F516EC0DF047
:1021B00004012C0E826FCBEC0AF03BC500F13CC54C
:1021C00001F13DC502F13EC503F10101000E046FAE
:1021D000000E056F010E066F000E076F39EC20F040
:1021E000A6EC20F02967F7EF10F0FCEF10F00401E7
:1021F0002D0E826FCBEC0AF030C182F40401300E58
:102200008227CBEC0AF031C182F40401300E822720
:10221000CBEC0AF004012E0E826FCBEC0AF032C137
:1022200082F40401300E8227CBEC0AF033C182F431
:102230000401300E8227CBEC0AF004012C0E826FD1
:10224000CBEC0AF003EC21F03FC500F140C501F1F1
:102250006CEC1BF004012C0E826FCBEC0AF003EC4B
:1022600021F041C500F1A6EC20F031C182F4040157
:10227000300E8227CBEC0AF032C182F40401300E1A
:102280008227CBEC0AF033C182F40401300E82279E
:10229000CBEC0AF0079455EF12F044EC21F085C323
:1022A0002AF186C32BF187C32CF188C32DF189C392
:1022B0002EF18AC32FF18BC330F18CC331F18DC362
:1022C00032F18EC333F10101296B51EC21F0C8ECDE
:1022D00020F00101010E046F000E056F000E066F65
:1022E000000E076F08EC20F0100E046F000E056F53
:1022F000000E066F000E076F19EC20F000C129F5E3
:1023000001C12AF502C12BF503C12CF571EC25F0B2
:1023100004014C0E826FCBEC0AF00401460E826F72
:10232000CBEC0AF004012C0E826FCBEC0AF025C531
:1023300000F126C501F127C502F128C503F101010D
:10234000100E046F000E056F000E066F000E076F73
:1023500039EC20F0A6EC20F02AC182F40401300E02
:102360008227CBEC0AF02BC182F40401300E8227C5
:10237000CBEC0AF02CC182F40401300E8227CBECA6
:102380000AF02DC182F40401300E8227CBEC0AF052
:102390002EC182F40401300E8227CBEC0AF02FC14B
:1023A00082F40401300E8227CBEC0AF030C182F4B3
:1023B0000401300E8227CBEC0AF031C182F4040113
:1023C000300E8227CBEC0AF032C182F40401300EC9
:1023D0008227CBEC0AF033C182F40401300E82274D
:1023E000CBEC0AF055EF12F00F9847EC26F042EFD5
:1023F0001AF004014C0E826FCBEC0AF00401350E8A
:10240000826FCBEC0AF004012C0E826FCBEC0AF049
:1024100003EC21F00784B5C500F10794A6EC20F089
:1024200031C182F40401300E8227CBEC0AF032C1B4
:1024300082F40401300E8227CBEC0AF033C182F41F
:102440000401300E8227CBEC0AF055EF12F00AECB3
:1024500026F003EC21F033C500F1A6EC20F00401D6
:102460004C0E826FCBEC0AF00401360E826FCBEC7F
:102470000AF004012C0E826FCBEC0AF031C182F419
:102480000401300E8227CBEC0AF032C182F4040141
:10249000300E8227CBEC0AF033C182F40401300EF7
:1024A0008227CBEC0AF055EF12F0D5EC0AF042EFA0
:1024B0001AF004014C0E826FCBEC0AF00401500EAE
:1024C000826FCBEC0AF004012C0E826FCBEC0AF089
:1024D00085C32AF186C32BF187C32CF188C32DF164
:1024E00089C32EF18AC32FF18BC330F18CC331F134
:1024F0008DC332F18EC333F1010151EC21F0C8ECF0
:1025000020F003018451530A0DE0030184514D0A68
:1025100038E00401780E826FCBEC0AF0D5EC0AF0BB
:1025200042EF1AF00401530E826FCBEC0AF0250E35
:102530000C6E00C10BF0A7EC07F0260E0C6E01C16B
:102540000BF0A7EC07F0270E0C6E02C10BF0A7EC06
:1025500007F0280E0C6E03C10BF0A7EC07F000C1CA
:1025600053F501C154F502C155F503C156F500C13B
:1025700057F501C158F502C159F503C15AF536EFB7
:1025800013F004014D0E826FCBEC0AF0290E0C6E95
:1025900000C10BF0A7EC07F000C15BF500C15CF5D2
:1025A00036EF13F004014C0E826FCBEC0AF00401FD
:1025B000540E826FCBEC0AF004012C0E826FCBEC30
:1025C0000AF084C32AF185C32BF186C32CF187C39B
:1025D0002DF188C32EF189C32FF18AC330F18BC34B
:1025E00031F18DC332F18EC333F1010151EC21F091
:1025F000C8EC20F00101000E046F000E056F010E03
:10260000066F000E076F19EC20F0210E0C6E00C152
:102610000BF0A7EC07F0220E0C6E01C10BF0A7EC3B
:1026200007F0230E0C6E02C10BF0A7EC07F0240E8E
:102630000C6E03C10BF0A7EC07F000C15DF501C102
:102640005EF502C15FF503C160F536EF13F00401DA
:102650004C0E826FCBEC0AF00401490E826FCBEC7A
:102660000AF004012C0E826FCBEC0AF0250EBEECB2
:1026700007F0E8CF00F1260EBEEC07F0E8CF01F13D
:10268000270EBEEC07F0E8CF02F1280EBEEC07F0F3
:10269000E8CF03F1A6EC20F089EC1EF00401730EE4
:1026A000826FCBEC0AF004012C0E826FCBEC0AF0A7
:1026B00003EC21F0290EBEEC07F0E8CF00F1A6EC08
:1026C00020F089EC1EF00401730E826FCBEC0AF04F
:1026D00004012C0E826FCBEC0AF057C500F158C5EF
:1026E00001F159C502F15AC503F1A6EC20F089ECBD
:1026F0001EF00401730E826FCBEC0AF004012C0E65
:10270000826FCBEC0AF003EC21F05CC500F1A6EC83
:1027100020F089EC1EF004016D0E826FCBEC0AF004
:1027200004012C0E826FCBEC0AF05DC500F15EC592
:1027300001F15FC502F160C503F15DEC1AF004011F
:102740002C0E826FCBEC0AF0D5EC0AF042EF1AF0B7
:1027500083C32AF184C32BF185C32CF186C32DF1E9
:1027600087C32EF188C32FF189C330F18AC331F1B9
:102770008BC332F18CC333F1010151EC21F0C8EC71
:1027800020F0160E0C6E00C10BF0A7EC07F0170E30
:102790000C6E01C10BF0A7EC07F0180E0C6E02C115
:1027A0000BF0A7EC07F0190E0C6E03C10BF0A7ECB1
:1027B00007F000C18AF101C18BF102C18CF103C1A4
:1027C0008DF100C18EF101C18FF102C190F103C101
:1027D00091F18AEF14F083C32AF184C32BF185C3EE
:1027E0002CF186C32DF187C32EF188C32FF189C345
:1027F00030F18AC331F18BC332F18CC333F1010163
:1028000051EC21F0C8EC20F000C18AF101C18BF13C
:1028100002C18CF103C18DF100C18EF101C18FF1B4
:1028200002C190F103C191F18AEF14F083C32AF140
:1028300084C32BF185C32CF186C32DF187C32EF100
:1028400088C32FF189C330F18AC331F18CC332F1CF
:102850008DC333F1010151EC21F0C8EC20F00101EE
:10286000000E046F000E056F010E066F000E076F5D
:1028700019EC20F01A0E0C6E00C10BF0A7EC07F05B
:102880001B0E0C6E01C10BF0A7EC07F01C0E0C6EBA
:1028900002C10BF0A7EC07F01D0E0C6E03C10BF08C
:1028A000A7EC07F000C192F101C193F102C194F1CC
:1028B00003C195F18AEF14F083C32AF184C32BF18D
:1028C00085C32CF186C32DF187C32EF188C32FF168
:1028D00089C330F18AC331F18CC332F18DC333F136
:1028E000010151EC21F0C8EC20F00101000E046F51
:1028F000000E056F010E066F000E076F19EC20F039
:1029000000C192F101C193F102C194F103C195F1AB
:102910008AEF14F0160EBEEC07F0E8CF00F1170EA8
:10292000BEEC07F0E8CF01F1180EBEEC07F0E8CFDF
:1029300002F1190EBEEC07F0E8CF03F1A6EC20F08F
:1029400089EC1EF00401730E826FCBEC0AF00401D7
:102950002C0E826FCBEC0AF08AC100F18BC101F121
:102960008CC102F18DC103F1A6EC20F089EC1EF0C0
:102970000401730E826FCBEC0AF004012C0E826FFF
:10298000CBEC0AF01A0EBEEC07F0E8CF00F11B0EFC
:10299000BEEC07F0E8CF01F11C0EBEEC07F0E8CF6B
:1029A00002F11D0EBEEC07F0E8CF03F15DEC1AF06A
:1029B00004012C0E826FCBEC0AF092C100F193C19E
:1029C00001F194C102F195C103F15DEC1AF0D5EC6F
:1029D0000AF042EF1AF00401690E826FCBEC0AF0A4
:1029E00004012C0E826FCBEC0AF00101040E006F83
:1029F000000E016F000E026F000E036FA6EC20F0B8
:102A00002CC182F40401300E8227CBEC0AF02DC1D8
:102A100082F40401300E8227CBEC0AF02EC182F43E
:102A20000401300E8227CBEC0AF02FC182F404019E
:102A3000300E8227CBEC0AF030C182F40401300E54
:102A40008227CBEC0AF031C182F40401300E8227D8
:102A5000CBEC0AF032C182F40401300E8227CBECB9
:102A60000AF033C182F40401300E8227CBEC0AF065
:102A700004012C0E826FCBEC0AF00101060E006FF0
:102A8000000E016F000E026F000E036FA6EC20F027
:102A90002CC182F40401300E8227CBEC0AF02DC148
:102AA00082F40401300E8227CBEC0AF02EC182F4AE
:102AB0000401300E8227CBEC0AF02FC182F404010E
:102AC000300E8227CBEC0AF030C182F40401300EC4
:102AD0008227CBEC0AF031C182F40401300E822748
:102AE000CBEC0AF032C182F40401300E8227CBEC29
:102AF0000AF033C182F40401300E8227CBEC0AF0D5
:102B000004012C0E826FCBEC0AF00101250E006F40
:102B1000000E016F000E026F000E036FA6EC20F096
:102B20002CC182F40401300E8227CBEC0AF02DC1B7
:102B300082F40401300E8227CBEC0AF02EC182F41D
:102B40000401300E8227CBEC0AF02FC182F404017D
:102B5000300E8227CBEC0AF030C182F40401300E33
:102B60008227CBEC0AF031C182F40401300E8227B7
:102B7000CBEC0AF032C182F40401300E8227CBEC98
:102B80000AF033C182F40401300E8227CBEC0AF044
:102B900004012C0E826FCBEC0AF0200EF86EF76A5F
:102BA000F66A04010900F5CF82F4CBEC0AF00900C3
:102BB000F5CF82F4CBEC0AF00900F5CF82F4CBEC30
:102BC0000AF00900F5CF82F4CBEC0AF00900F5CF4A
:102BD00082F4CBEC0AF00900F5CF82F4CBEC0AF0DA
:102BE0000900F5CF82F4CBEC0AF00900F5CF82F4AE
:102BF000CBEC0AF0D5EC0AF042EF1AF08351630AED
:102C0000D8A442EF1AF08451610AD8A442EF1AF016
:102C100085516C0AD8A442EF1AF08651410A42E06D
:102C20008651440A1BE08651420AD8B465EF16F07B
:102C30008651350AD8B4CCEF1BF08651360AD8B489
:102C400021EF1CF08651370AD8B48AEF1CF0865168
:102C5000380AD8B4E8EF1CF042EF1AF00798079A48
:102C600004017A0E826FCBEC0AF00401780E826FB9
:102C7000CBEC0AF00401640E826FCBEC0AF081A861
:102C800049EF16F00401550E826FCBEC0AF04EEFBF
:102C900016F004014C0E826FCBEC0AF0D5EC0AF072
:102CA00042EF1AF00788079A04017A0E826FCBEC84
:102CB0000AF00401410E826FCBEC0AF00401610EB0
:102CC000826FCBEC0AF03FEF16F00798078A0401F9
:102CD0007A0E826FCBEC0AF00401420E826FCBECCD
:102CE0000AF00401610E826FCBEC0AF03FEF16F0A0
:102CF0000101666783EF16F0676783EF16F0686778
:102D000083EF16F069679BEF16F04F678FEF16F0B1
:102D100050678FEF16F051678FEF16F052679BEFF9
:102D200016F00101000E006F000E016F000E026F21
:102D3000000E036F12000101620E046F010E056F99
:102D4000000E066F000E076F66C100F167C101F14A
:102D500068C102F169C103F108EC20F003BF1FEF65
:102D600017F00101000E046FA80E056F550E066FD7
:102D7000020E076F66C100F167C101F168C102F17F
:102D800069C103F166C186F167C187F168C188F145
:102D900069C189F108EC20F003BFD8EF16F00101FA
:102DA000000E866FA80E876F550E886F020E896F12
:102DB0000E0EBEEC07F0E8CF18F10F0EBEEC07F0D8
:102DC000E8CF19F1100EBEEC07F0E8CF1AF1110EA2
:102DD000BEEC07F0E8CF1BF151EC1FF086C104F107
:102DE00087C105F188C106F189C107F108EC20F01F
:102DF000078215EC1FF051EC1FF0079215EC1FF045
:102E000086C100F187C101F188C102F189C103F1D6
:102E1000079215EC1FF0CC0E046FE00E056F870EC5
:102E2000066F050E076F08EC20F000C118F101C114
:102E300019F102C11AF103C11BF157EF17F001019B
:102E4000800E006F1A0E016F060E026F000E036FE8
:102E50004FC104F150C105F151C106F152C107F152
:102E600008EC20F003AF38EF17F003EC21F012006C
:102E70000E0EBEEC07F0E8CF18F10F0EBEEC07F017
:102E8000E8CF19F1100EBEEC07F0E8CF1AF1110EE1
:102E9000BEEC07F0E8CF1BF14FC100F150C101F1CA
:102EA00051C102F152C103F1078215EC1FF018C1A4
:102EB00000F119C101F11AC102F11BC103F11200A5
:102EC0000401730E826FCBEC0AF004012C0E826FAA
:102ED000CBEC0AF0078462C166F163C167F164C19B
:102EE00068F165C169F14BC14FF14CC150F14DC161
:102EF00051F14EC152F157C159F158C15AF10794DD
:102F000086EC17F0D5EC0AF042EF1AF066C100F13A
:102F100067C101F168C102F169C103F10101A6ECC9
:102F200020F089EC1EF00401630E826FCBEC0AF0F6
:102F300004012C0E826FCBEC0AF04FC100F150C19E
:102F400001F151C102F152C103F10101A6EC20F0DF
:102F500089EC1EF00401660E826FCBEC0AF00401CE
:102F60002C0E826FCBEC0AF003EC21F059C100F17A
:102F70005AC101F10101A6EC20F089EC1EF0040118
:102F8000740E826FCBEC0AF0120010820401530E13
:102F9000826FCBEC0AF004012C0E826FCBEC0AF0AE
:102FA00083C32AF184C32BF185C32CF186C32DF191
:102FB00087C32EF188C32FF189C330F18AC331F161
:102FC0008BC332F18CC333F1010151EC21F0C8EC19
:102FD00020F000C166F101C167F102C168F103C1CF
:102FE00069F18EC32AF18FC32BF190C32CF191C3E9
:102FF0002DF192C32EF193C32FF194C330F195C3F9
:1030000031F196C332F197C333F1010151EC21F054
:10301000C8EC20F000C14FF101C150F102C151F1E3
:1030200003C152F144EC21F099C32FF19AC330F15E
:103030009BC331F19CC332F19DC333F1010151ECCB
:1030400021F0C8EC20F000C159F101C15AF186EC21
:1030500017F004012C0E826FCBEC0AF037EF18F05A
:103060008251520A03E10F8237EF18F00F9282511A
:10307000750A03E110843EEF18F010948251550A4E
:1030800003E1108645EF18F01096078410B2A2EF06
:1030900018F010A48EEF18F0B6C166F1B7C167F151
:1030A000B8C168F1B9C169F1BAC16AF1BBC16BF1CC
:1030B000BCC16CF1BDC16DF1BEC16EF1BFC16FF19C
:1030C000C0C170F1C1C171F1C2C172F1C3C173F16C
:1030D000C4C174F1C5C175F1C6C176F1C7C177F13C
:1030E000C8C178F1C9C179F1CAC17AF1CBC17BF10C
:1030F000CCC17CF1CDC17DF1CEC17EF1CFC17FF1DC
:10310000D0C180F1D1C181F1D2C182F1D3C183F1AB
:10311000D4C184F1D5C185F196EF18F062C166F192
:1031200063C167F164C168F165C169F14BC14FF1D9
:103130004CC150F14DC151F14EC152F157C159F13D
:1031400058C15AF107940FA0C4EF18F0010192671B
:10315000B1EF18F09367B1EF18F09467B1EF18F082
:103160009567B5EF18F0C4EF18F078EC16F092C13F
:1031700004F193C105F194C106F195C107F108EC82
:1031800020F003BF08EF1AF078EC16F00101000EF2
:10319000046F000E056F010E066F000E076F39EC0D
:1031A00020F010A4DBEF18F00401750E826FCBEC59
:1031B0000AF0E0EF18F00401720E826FCBEC0AF017
:1031C00004012C0E826FCBEC0AF0A6EC20F02967EC
:1031D000EFEF18F00401200E826FF2EF18F00401F7
:1031E0002D0E826FCBEC0AF030C182F40401300E58
:1031F0008227CBEC0AF031C182F40401300E822721
:10320000CBEC0AF004012E0E826FCBEC0AF032C137
:1032100082F40401300E8227CBEC0AF033C182F431
:103220000401300E8227CBEC0AF004016D0E826F90
:10323000CBEC0AF004012C0E826FCBEC0AF04FC1EC
:1032400000F150C101F151C102F152C103F101017C
:10325000A6EC20F089EC1EF00401480E826FCBEC46
:103260000AF004017A0E826FCBEC0AF004012C0EF6
:10327000826FCBEC0AF066C100F167C101F168C151
:1032800002F169C103F10101A6EC20F089EC1EF006
:103290000401630E826FCBEC0AF004012C0E826FE6
:1032A000CBEC0AF066C100F167C101F168C102F11F
:1032B00069C103F101010A0E046F000E056F000ED3
:1032C000066F000E076F19EC20F0000E046F120E4F
:1032D000056F000E066F000E076F39EC20F0A6ECAC
:1032E00020F02AC182F40401300E8227CBEC0AF0D0
:1032F0002BC182F40401300E8227CBEC0AF02CC1E2
:1033000082F40401300E8227CBEC0AF02DC182F446
:103310000401300E8227CBEC0AF02EC182F40401A6
:10332000300E8227CBEC0AF02FC182F40401300E5C
:103330008227CBEC0AF030C182F40401300E8227E0
:10334000CBEC0AF004012E0E826FCBEC0AF031C1F7
:1033500082F40401300E8227CBEC0AF032C182F4F1
:103360000401300E8227CBEC0AF033C182F4040151
:10337000300E8227CBEC0AF00401730E826FCBEC87
:103380000AF004012C0E826FCBEC0AF003EC21F062
:1033900059C100F15AC101F16CEC1BF00FB2D4EF2E
:1033A00019F00FA006EF1AF004012C0E826FCBEC7F
:1033B0000AF0200EF86EF76AF66A04010900F5CFEC
:1033C00082F4CBEC0AF00900F5CF82F4CBEC0AF0E2
:1033D0000900F5CF82F4CBEC0AF00900F5CF82F4B6
:1033E000CBEC0AF00900F5CF82F4CBEC0AF009002F
:1033F000F5CF82F4CBEC0AF00900F5CF82F4CBECE8
:103400000AF00900F5CF82F4CBEC0AF0D5EC0AF013
:103410000F9042EF1AF00401630E826FCBEC0AF0BA
:1034200004012C0E826FCBEC0AF048EC1AF0040178
:103430002C0E826FCBEC0AF0BBEC1AF004012C0EC0
:10344000826FCBEC0AF037EC1BF004012C0E826F7C
:10345000CBEC0AF00101F80E006FCD0E016F660E85
:10346000026F030E036F5DEC1AF004012C0E826FE5
:10347000CBEC0AF04DEC1BF0D5EC0AF042EF1AF061
:10348000D5EC0AF00301C26B0790109251EF1DF0CA
:10349000D8900E0EBEEC07F0E8CF00F10F0EBEEC98
:1034A00007F0E8CF01F1100EBEEC07F0E8CF02F113
:1034B000110EBEEC07F0E8CF03F10101000E046F1E
:1034C000000E056F010E066F000E076F39EC20F03D
:1034D000A6EC20F02AC182F40401300E8227CBEC46
:1034E0000AF02BC182F40401300E8227CBEC0AF0E3
:1034F0002CC182F40401300E8227CBEC0AF02DC1DE
:1035000082F40401300E8227CBEC0AF02EC182F443
:103510000401300E8227CBEC0AF02FC182F40401A3
:10352000300E8227CBEC0AF030C182F40401300E59
:103530008227CBEC0AF031C182F40401300E8227DD
:10354000CBEC0AF004012E0E826FCBEC0AF032C1F4
:1035500082F40401300E8227CBEC0AF033C182F4EE
:103560000401300E8227CBEC0AF004016D0E826F4D
:10357000CBEC0AF01200120EBEEC07F0E8CF00F11F
:10358000130EBEEC07F0E8CF01F1140EBEEC07F00D
:10359000E8CF02F1150EBEEC07F0E8CF03F1010110
:1035A0000A0E046F000E056F000E066F000E076F07
:1035B00019EC20F0000E046F120E056F000E066F5E
:1035C000000E076F39EC20F0A6EC20F02AC182F43F
:1035D0000401300E8227CBEC0AF02BC182F40401E7
:1035E000300E8227CBEC0AF02CC182F40401300E9D
:1035F0008227CBEC0AF02DC182F40401300E822721
:10360000CBEC0AF02EC182F40401300E8227CBEC01
:103610000AF02FC182F40401300E8227CBEC0AF0AD
:1036200030C182F40401300E8227CBEC0AF0040191
:103630002E0E826FCBEC0AF031C182F40401300E01
:103640008227CBEC0AF032C182F40401300E8227CB
:10365000CBEC0AF033C182F40401300E8227CBECAC
:103660000AF00401730E826FCBEC0AF012000A0E0E
:10367000BEEC07F0E8CF00F10B0EBEEC07F0E8CF90
:1036800001F10C0EBEEC07F0E8CF02F10D0EBEEC1E
:1036900007F0E8CF03F16CEF1BF0060EBEEC07F06D
:1036A000E8CF00F1070EBEEC07F0E8CF01F1080EFD
:1036B000BEEC07F0E8CF02F1090EBEEC07F0E8CF50
:1036C00003F16CEF1BF0010103EC21F0078457C1FB
:1036D00000F158C101F107940101E80E046F800E5A
:1036E000056F000E066F000E076F19EC20F0000E3C
:1036F000046F040E056F000E066F000E076F39ECA5
:1037000020F0880E046F130E056F000E066F000E7A
:10371000076F08EC20F00A0E046F000E056F000E14
:10372000066F000E076F39EC20F0A6EC20F00101C7
:103730002967A0EF1BF00401200E826FA3EF1BF09E
:1037400004012D0E826FCBEC0AF030C182F404012B
:10375000300E8227CBEC0AF031C182F40401300E26
:103760008227CBEC0AF032C182F40401300E8227AA
:10377000CBEC0AF004012E0E826FCBEC0AF033C1C1
:1037800082F40401300E8227CBEC0AF00401430ED0
:10379000826FCBEC0AF0120087C32AF188C32BF1A9
:1037A00089C32CF18AC32DF18BC32EF18CC32FF169
:1037B0008DC330F18EC331F190C332F191C333F137
:1037C0000101296B51EC21F0C8EC20F00101000E41
:1037D000046F000E056F010E066F000E076F19ECE7
:1037E00020F00E0E0C6E00C10BF0A7EC07F00F0ED0
:1037F0000C6E01C10BF0A7EC07F0100E0C6E02C1AD
:103800000BF0A7EC07F0110E0C6E03C10BF0A7EC48
:1038100007F004017A0E826FCBEC0AF004012C0E43
:10382000826FCBEC0AF00401350E826FCBEC0AF00C
:1038300004012C0E826FCBEC0AF048EC1AF04EEF2C
:1038400016F087C32AF188C32BF189C32CF18AC3F0
:103850002DF18BC32EF18CC32FF18DC330F18EC3AC
:1038600031F190C332F191C333F10101296B51EC75
:1038700021F0C8EC20F0880E046F130E056F000EC7
:10388000066F000E076F0DEC20F0000E046F040EA3
:10389000056F000E066F000E076F19EC20F0010196
:1038A000E80E046F800E056F000E066F000E076FA6
:1038B00039EC20F00A0E0C6E00C10BF0A7EC07F0FB
:1038C0000B0E0C6E01C10BF0A7EC07F00C0E0C6E8A
:1038D00002C10BF0A7EC07F00D0E0C6E03C10BF04C
:1038E000A7EC07F004017A0E826FCBEC0AF004011A
:1038F0002C0E826FCBEC0AF00401360E826FCBECFB
:103900000AF004012C0E826FCBEC0AF037EC1BF0AE
:103910004EEF16F087C32AF188C32BF189C32CF12F
:103920008AC32DF18BC32EF18CC32FF18DC330F1DF
:103930008FC331F190C332F191C333F1010151ECE6
:1039400021F0C8EC20F0000E046F120E056F000E7F
:10395000066F000E076F19EC20F001010A0E046FCC
:10396000000E056F000E066F000E076F39EC20F099
:10397000120E0C6E00C10BF0A7EC07F0130E0C6ECC
:1039800001C10BF0A7EC07F0140E0C6E02C10BF096
:10399000A7EC07F0150E0C6E03C10BF0A7EC07F0B7
:1039A00004017A0E826FCBEC0AF004012C0E826FB8
:1039B000CBEC0AF00401370E826FCBEC0AF0040165
:1039C0002C0E826FCBEC0AF0BBEC1AF04EEF16F027
:1039D00087C32AF188C32BF189C32CF18AC32DF147
:1039E0008BC32EF18CC32FF18DC330F18EC331F117
:1039F00090C332F191C333F10101296B51EC21F0F5
:103A0000C8EC20F0880E046F130E056F000E066FD1
:103A1000000E076F0DEC20F0000E046F040E056F12
:103A2000000E066F000E076F19EC20F00101E80E82
:103A3000046F800E056F000E066F000E076F39ECE5
:103A400020F0060E0C6E00C10BF0A7EC07F0070E7D
:103A50000C6E01C10BF0A7EC07F0080E0C6E02C152
:103A60000BF0A7EC07F0090E0C6E03C10BF0A7ECEE
:103A700007F004017A0E826FCBEC0AF004012C0EE1
:103A8000826FCBEC0AF00401380E826FCBEC0AF0A7
:103A900004012C0E826FCBEC0AF04DEC1BF04EEFC4
:103AA00016F081A80FEF1EF007A8C8EF1DF0010166
:103AB000800E006F1A0E016F060E026F000E036F6C
:103AC0004BC104F14CC105F14DC106F14EC107F1E6
:103AD00008EC20F003BF0FEF1EF083EC1EF04BC18B
:103AE00000F14CC101F14DC102F14EC103F1078259
:103AF00015EC1FF018C104F119C105F11AC106F146
:103B00001BC107F1F80E006FCD0E016F660E026F3C
:103B1000030E036F08EC20F00E0E0C6E00C10BF0CC
:103B2000A7EC07F00F0E0C6E01C10BF0A7EC07F02D
:103B3000100E0C6E02C10BF0A7EC07F0110E0C6E0C
:103B400003C10BF0A7EC07F00784010103EC21F09F
:103B500057C100F158C101F107940A0E0C6E00C163
:103B60000BF0A7EC07F00B0E0C6E01C10BF0A7ECED
:103B700007F00C0E0C6E02C10BF0A7EC07F00D0E57
:103B80000C6E03C10BF0A7EC07F007980FEF1EF0C7
:103B900007AA0FEF1EF00784010103EC21F057C1C3
:103BA00000F158C101F10794060E0C6E00C10BF034
:103BB000A7EC07F0070E0C6E01C10BF0A7EC07F0A5
:103BC000080E0C6E02C10BF0A7EC07F0090E0C6E8C
:103BD00003C10BF0A7EC07F0078462C100F163C1D9
:103BE00001F164C102F165C103F10794120E0C6E7C
:103BF00000C10BF0A7EC07F0130E0C6E01C10BF027
:103C0000A7EC07F0140E0C6E02C10BF0A7EC07F046
:103C1000150E0C6E03C10BF0A7EC07F0079A040118
:103C2000805181197F0B0BE09EA809D014EE00F0A3
:103C300081517F0BE126E750812B0F01AD6E05010D
:103C40002F51010A13E081AA36EF1EF005012F5112
:103C5000000A0AE00FB836EF1EF00501306736EFB4
:103C60001EF00FB836EF1EF0CFEF27F081B84BEF04
:103C70001EF02DEC22F005012F51020A02E04BEF5D
:103C80001EF05C2F4BEF1EF05BC55CF50501010ECD
:103C9000306F3C0E316F2FEF0AF018C100F119C1DF
:103CA00001F11AC102F11BC103F1000E046F000EF5
:103CB000056F010E066F000E076F39EC20F029A189
:103CC00078EF1EF02051D8B478EF1EF018C100F143
:103CD00019C101F11AC102F11BC103F1000E046FF9
:103CE000000E056F0A0E066F000E076F39EC20F00C
:103CF0001200010104510013055101130651021372
:103D00000751031312000101186B196B1A6B1B6B1F
:103D100012002AC182F40401300E8227CBEC0AF093
:103D20002BC182F40401300E8227CBEC0AF02CC1A7
:103D300082F40401300E8227CBEC0AF02DC182F40C
:103D40000401300E8227CBEC0AF02EC182F404016C
:103D5000300E8227CBEC0AF02FC182F40401300E22
:103D60008227CBEC0AF030C182F40401300E8227A6
:103D7000CBEC0AF031C182F40401300E8227CBEC87
:103D80000AF032C182F40401300E8227CBEC0AF033
:103D900033C182F40401300E8227CBEC0AF012000A
:103DA0002FC182F40401300E8227CBEC0AF030C11F
:103DB00082F40401300E8227CBEC0AF031C182F488
:103DC0000401300E8227CBEC0AF032C182F40401E8
:103DD000300E8227CBEC0AF033C182F40401300E9E
:103DE0008227CBEC0AF01200060E116E060E126E40
:103DF000060E136E112EFAEF1EF0122EFAEF1EF0C1
:103E0000132EFAEF1EF08B84020E116E020E126E4C
:103E1000020E136E112E0AEF1FF0122E0AEF1FF082
:103E2000132E0AEF1FF08B9412000101005305E1DD
:103E3000015303E1025301E1002BD8EC1FF003EC26
:103E400021F03951006F3A51016F420E046F4B0E51
:103E5000056F000E066F000E076F19EC20F000C111
:103E600004F101C105F102C106F103C107F118C156
:103E700000F119C101F11AC102F11BC103F107B22E
:103E800046EF1FF00DEC20F048EF1FF008EC20F09B
:103E900000C118F101C119F102C11AF103C11BF1EE
:103EA000120003EC21F059C100F15AC101F1060ED4
:103EB000BEEC07F0E8CF04F1070EBEEC07F0E8CF48
:103EC00005F1080EBEEC07F0E8CF06F1090EBEECD6
:103ED00007F0E8CF07F108EC20F000C124F101C1A0
:103EE00025F102C126F103C127F1290E046F000E4E
:103EF000056F000E066F000E076F19EC20F0EE0E36
:103F0000046F430E056F000E066F000E076F0DEC79
:103F100020F024C104F125C105F126C106F127C115
:103F200007F119EC20F000C11CF101C11DF102C123
:103F30001EF103C11FF1120EBEEC07F0E8CF04F131
:103F4000130EBEEC07F0E8CF05F1140EBEEC07F03F
:103F5000E8CF06F1150EBEEC07F0E8CF07F10D0E25
:103F6000006F000E016F000E026F000E036F19EC60
:103F700020F0180E046F000E056F000E066F000E85
:103F8000076F39EC20F01CC104F11DC105F11EC101
:103F900006F11FC107F10DEC20F06A0E046F2A0E26
:103FA000056F000E066F000E076F08EC20F0120080
:103FB000BF0EFA6E200E3A6F396BD890003701377A
:103FC00002370337D8B0E9EF1FF03A2FDEEF1FF0CA
:103FD00039073A070353D8B412000331070B80099D
:103FE0003F6F03390F0B010F396F80EC5FF0406FAB
:103FF000390580EC5FF0405D405F396B3F33D8B0EE
:10400000392739333FA9FEEF1FF0405139271200FD
:10401000010128EC21F0D8B0120001010351071969
:10402000346FEBEC20F0D8900751031934AF800FB8
:1040300012000101346B0FEC21F0D8A025EC21F027
:10404000D8B01200FAEC20F003EC21F01F0E366F0E
:104050003BEC21F00B35D8B0EBEC20F0D8A00335C9
:10406000D8B01200362F28EF20F034B112EC21F036
:1040700012000101346B04510511061107110008EB
:10408000D8A00FEC21F0D8A025EC21F0D8B0120078
:10409000086B096B0A6B0B6B3BEC21F01F0E366F44
:1040A0003BEC21F007510B5DD8A463EF20F00651E3
:1040B0000A5DD8A463EF20F00551095DD8A463EF31
:1040C00020F00451085DD8A076EF20F00451085F7D
:1040D0000551D8A0053D095F0651D8A0063D0A5FED
:1040E0000751D8A0073D0B5FD8900081362F50EFC5
:1040F00020F034B112EC21F0346B0FEC21F0D890A9
:104100003FEC21F007510B5DD8A493EF20F006514E
:104110000A5DD8A493EF20F00551095DD8A493EF70
:1041200020F00451085DD8A0A2EF20F0003FA2EFDC
:1041300020F0013FA2EF20F0023FA2EF20F0032B7E
:10414000D8B4120034B112EC21F012000101346B2A
:104150000FEC21F0D8B0120044EC21F0200E366FA5
:10416000003701370237033711EE33F00A0E376F8D
:10417000E7360A0EE75CD8B0E76EE552372FB8EFA6
:1041800020F0362FB0EF20F034B12981D890120002
:1041900001010A0E346F200E366F11EE29F03451F2
:1041A000376F0A0ED890E652D8B0E726E732372F9D
:1041B000D3EF20F00333023301330033362FCDEF3A
:1041C00020F0E750FF0FD8A00335D8B0120029B176
:1041D00012EC21F01200045100270551D8B0053D22
:1041E00001270651D8B0063D02270751D8B0073D38
:1041F000032712000051086F0151096F02510A6F25
:1042000003510B6F12000101006B016B026B036B1A
:1042100012000101046B056B066B076B120003357E
:10422000D8A012000351800B001F011F021F031FA3
:10423000003F22EF21F0013F22EF21F0023F22EF69
:1042400021F0032B342B032512000735D8A01200D0
:104250000751800B041F051F061F071F043F38EF7F
:1042600021F0053F38EF21F0063F38EF21F0072B12
:10427000342B072512000037013702370337083780
:1042800009370A370B3712000101296B2A6B2B6B98
:104290002C6B2D6B2E6B2F6B306B316B326B336B4A
:1042A000120001012A510F0B2A6F2B510F0B2B6F9C
:1042B0002C510F0B2C6F2D510F0B2D6F2E510F0BFF
:1042C0002E6F2F510F0B2F6F30510F0B306F31515D
:1042D0000F0B316F32510F0B326F33510F0B336FA6
:1042E0001200000EC76E220EC66E10A802D089946E
:1042F00012008984120010A802D0898412008994C7
:10430000120071EC21F09E96C69E000EC96EFF0E43
:104310009EB602D0E82EFCD79E96C69E000EC96EB1
:10432000FF0E9EB602D0E82EFCD7C9CFABF59E9605
:10433000C69E000EC96EFF0E9EB602D0E82EFCD7B8
:10434000C9CFACF59E96C69E000EC96EFF0E9EB6F6
:1043500002D0E82EFCD7C9CFADF59E96C69E000EC2
:10436000C96EFF0E9EB602D0E82EFCD7C9CFAEF5BF
:104370009E96C69E000EC96EFF0E9EB602D0E82E17
:10438000FCD7C9CFAFF59E96C69E000EC96EFF0E34
:104390009EB602D0E82EFCD7C9CFB0F59E96C69E39
:1043A000000EC96EFF0E9EB602D0E82EFCD7C9CF14
:1043B000B1F57BEC21F00FEC24F0120071EC21F050
:1043C0009E96C69E800EC96EFF0E9EB602D0E82E47
:1043D000FCD79E96C69EABC5C9FFFF0E9EB602D007
:1043E000E82EFCD79E96C69EACC5C9FFFF0E9EB6B2
:1043F00002D0E82EFCD79E96C69EADC5C9FFFF0E23
:104400009EB602D0E82EFCD79E96C69EAEC5C9FFCA
:10441000FF0E9EB602D0E82EFCD79E96C69EAFC574
:10442000C9FFFF0E9EB602D0E82EFCD79E96C69E10
:10443000B0C5C9FFFF0E9EB602D0E82EFCD79E96EF
:10444000C69EB1C5C9FFFF0E9EB602D0E82EFCD7AE
:104450007BEC21F00FEC24F0120071EC21F09E9621
:10446000C69E070EC96EFF0E9EB602D0E82EFCD780
:104470009E96C69E000EC96EFF0E9EB602D0E82E16
:10448000FCD7C9CFABF59E96C69E000EC96EFF0E37
:104490009EB602D0E82EFCD7C9CFACF59E96C69E3C
:1044A000000EC96EFF0E9EB602D0E82EFCD7C9CF13
:1044B000ADF59E96C69E000EC96EFF0E9EB602D04A
:1044C000E82EFCD7C9CFAEF57BEC21F00FEC24F041
:1044D00071EC21F09E96C69E0E0EC96EFF0E9EB622
:1044E00002D0E82EFCD79E96C69E000EC96EFF0E27
:1044F0009EB602D0E82EFCD7C9CFB2F57BEC21F0F6
:104500000FEC24F0120071EC21F09E96C69E870EEF
:10451000C96EFF0E9EB602D0E82EFCD79E96C69EB0
:10452000ABC5C9FFFF0E9EB602D0E82EFCD79E9603
:10453000C69EACC5C9FFFF0E9EB602D0E82EFCD7C2
:104540009E96C69EADC5C9FFFF0E9EB602D0E82E50
:10455000FCD79E96C69EAEC5C9FFFF0E9EB602D082
:10456000E82EFCD77BEC21F00FEC24F071EC21F06D
:104570009E96C69E16C0C9FFFF0E9EB602D0E82EBC
:10458000FCD79E96C69EB3C5C9FFFF0E9EB602D04D
:10459000E82EFCD77BEC21F00FEC24F0120071EC3C
:1045A00021F09E96C69E870EC96EFF0E9EB602D063
:1045B000E82EFCD79E96C69E000EC96EFF0E9EB6D4
:1045C00002D0E82EFCD79E96C69E800EC96EFF0EC6
:1045D0009EB602D0E82EFCD79E96C69E800EC96E6F
:1045E000FF0E9EB602D0E82EFCD79E96C69E800E89
:1045F000C96EFF0E9EB602D0E82EFCD77BEC21F0F0
:104600000FEC24F0120071EC21F09E96C69E870EEE
:10461000C96EFF0E9EB602D0E82EFCD79E96C69EAF
:10462000000EC96EFF0E9EB602D0E82EFCD79E96F5
:10463000C69E000EC96EFF0E9EB602D0E82EFCD7B5
:104640009E96C69E800EC96EFF0E9EB602D0E82EC4
:10465000FCD79E96C69E800EC96EFF0E9EB602D0F7
:10466000E82EFCD77BEC21F00FEC24F0120010A810
:1046700035D071EC21F09E96C69E16C0C9FFFF0E84
:104680009EB602D0E82EFCD70FEC24F09E96C69E74
:10469000450EC96EFF0E9EB602D0E82EFCD77BEC0D
:1046A00021F00FEC24F071EC21F09E96C69E8F0E47
:1046B000C96EFF0E9EB602D0E82EFCD70FEC24F098
:1046C0009E96C69E000EC96EFF0E9EB602D0E82EC4
:1046D000FCD77BEC21F00FEC24F0120071EC21F000
:1046E0009E96C69E16C0C9FFFF0E9EB602D0E82E4B
:1046F000FCD70FEC24F09E96C69E010EC96EFF0EED
:104700009EB602D0E82EFCD77BEC21F00FEC24F013
:1047100071EC21F09E96C69E910EC96EFF0E9EB65C
:1047200002D0E82EFCD70FEC24F09E96C69EA50E74
:10473000C96EFF0E9EB602D0E82EFCD77BEC21F0AE
:104740000FEC24F0120071EC21F09E96C69E16C06C
:10475000C9FFFF0E9EB602D0E82EFCD70FEC24F066
:104760009E96C69E810EC96EFF0E9EB602D0E82EA2
:10477000FCD77BEC21F00FEC24F0120071EC21F05F
:104780009E96C69E16C0C9FFFF0E9EB602D0E82EAA
:10479000FCD70FEC24F09E96C69E010EC96EFF0E4C
:1047A0009EB602D0E82EFCD77BEC21F00FEC24F073
:1047B000120071EC21F09E96C69E910EC96EFF0EFE
:1047C0009EB602D0E82EFCD70FEC24F09E96C69E33
:1047D000A50EC96EFF0E9EB602D0E82EFCD77BEC6C
:1047E00021F00FEC24F0120071EC21F09E96C69E91
:1047F000910EC96EFF0E9EB602D0E82EFCD70FECCC
:1048000024F09E96C69E000EC96EFF0E9EB602D084
:10481000E82EFCD77BEC21F00FEC24F01200050E03
:10482000E82EFED712000501256B266B276B286B3F
:10483000899A400EC76E200EC66E9E96C69E030EC7
:10484000C96EFF0E9EB602D0E82EFCD79E96C69E7D
:1048500027C5C9FFFF0E9EB602D0E82EFCD79E9654
:10486000C69E26C5C9FFFF0E9EB602D0E82EFCD715
:104870009E96C69E25C5C9FFFF0E9EB602D0E82EA5
:10488000FCD79E96C69EC952FF0E9EB602D0E82E59
:10489000FCD7898A0F01C950FF0A01E11200050106
:1048A0002E51130A05E005012E51170A0CE01200E3
:1048B0000501F00E256FFF0E266F0F0E276F000EFD
:1048C000286F6CEF24F00501F00E256FFF0E266FA8
:1048D000FF0E276F000E286F899A400EC76E200EBC
:1048E000C66E9E96C69E030EC96EFF0E9EB602D081
:1048F000E82EFCD79E96C69E27C5C9FFFF0E9EB622
:1049000002D0E82EFCD79E96C69E26C5C9FFFF0E94
:104910009EB602D0E82EFCD79E96C69E25C5C9FF3E
:10492000FF0E9EB602D0E82EFCD79E96C69EC952B8
:10493000FF0E9EB602D0E82EFCD7898A0F01C9501F
:10494000FF0A1DE005012E51130A05E005012E5155
:10495000170A0BE012000501000E256F000E266FEE
:10496000100E276F000E286F12000501000E256F34
:10497000000E266F000E276F010E286F1200050132
:10498000256B266B276B286B05012E51130A05E05A
:1049900005012E51170A0CE012000501000E216FCF
:1049A000000E226F080E236F000E246FE1EF24F03B
:1049B0000501000E216F000E226F800E236F000E86
:1049C000246F21C500F122C501F123C502F124C5E0
:1049D00003F125C504F126C505F127C506F128C553
:1049E00007F179EC1EF000C125F501C126F502C1E1
:1049F00027F503C128F5899A400EC76E200EC66EB2
:104A00009E96C69E030EC96EFF0E9EB602D0E82E7D
:104A1000FCD79E96C69E27C5C9FFFF0E9EB602D044
:104A2000E82EFCD79E96C69E26C5C9FFFF0E9EB6F1
:104A300002D0E82EFCD79E96C69E25C5C9FFFF0E64
:104A40009EB602D0E82EFCD79E96C69EC952FF0E97
:104A50009EB602D0E82EFCD7898AC950FF0A08E129
:104A600004C125F505C126F506C127F507C128F5BE
:104A7000D890050124332333223321332151F00B05
:104A8000216F21674BEF25F022674BEF25F023675D
:104A90004BEF25F02467E1EF24F00501100E2527E8
:104AA000E86A2623E86A2723E86A28231200E86ACE
:104AB00005012E51130A06E005012E51170A0BE0DD
:104AC000020E120005012851000A03E12751F00BE4
:104AD00007E0010E120005012851000A01E0010E55
:104AE000120029C500F12AC501F12BC502F12CC520
:104AF00003F125C504F126C505F127C506F128C532
:104B000007F108EC20F003BF120057EC25F0D8A401
:104B1000E9EF25F0899A400EC76E200EC66E9E966C
:104B2000C69E060EC96EFF0E9EB602D0E82EFCD7BA
:104B3000898A899A9E96C69E020EC96EFF0E9EB6FF
:104B400002D0E82EFCD79E96C69E27C5C9FFFF0E51
:104B50009EB602D0E82EFCD79E96C69E26C5C9FFFB
:104B6000FF0E9EB602D0E82EFCD79E96C69E25C5A7
:104B7000C9FFFF0E9EB602D0E82EFCD79E96C69EB9
:104B8000000EC96EFF0E9EB602D0E82EFCD7898AB1
:104B9000899A9E96C69E050EC96EFF0E9EB602D0DD
:104BA000E82EFCD79E96C69EC952FF0E9EB602D036
:104BB000E82EFCD7C9B0D2EF25F0898A0501100E86
:104BC0002527E86A2623E86A2723E86A282371EF65
:104BD00025F01200899A400EC76E200EC66E9E9672
:104BE000C69E060EC96EFF0E9EB602D0E82EFCD7FA
:104BF000898A899A9E96C69EC70EC96EFF0E9EB67A
:104C000002D0E82EFCD7898A0501256B266B276B1D
:104C1000286B1200899A400EC76E200EC66E9E96B3
:104C2000C69E050EC96EFF0E9EB602D0E82EFCD7BA
:104C30009E96C69EC952FF0E9EB602D0E82EFCD7A5
:104C4000C9CF33F5898A1200899A400EC76E200EAB
:104C5000C66E9E96C69EB90EC96EFF0E9EB602D057
:104C6000E82EFCD7898A1200899A400EC76E200E62
:104C7000C66E9E96C69EAB0EC96EFF0E9EB602D045
:104C8000E82EFCD7898AFF0EE82EFED7120057ECDB
:104C900025F0D8A41200899A400EC76E200EC66E69
:104CA0009E96C69E030EC96EFF0E9EB602D0E82EDB
:104CB000FCD79E96C69E27C5C9FFFF0E9EB602D0A2
:104CC000E82EFCD79E96C69E26C5C9FFFF0E9EB64F
:104CD00002D0E82EFCD79E96C69E25C5C9FFFF0EC2
:104CE0009EB602D0E82EFCD79E96C69EC952FF0EF5
:104CF0009EB602D0E82EFCD7898A0F01C950FF0A60
:104D0000D8A442EF27F00501FE0E336F81EC21F0AD
:104D1000ABC534F5ACC535F5ADC536F5AEC537F523
:104D2000AFC538F5B0C539F5B1C53AF50784B6C198
:104D300066F1B7C167F1B8C168F1B9C169F14BC19A
:104D40004FF14CC150F14DC151F14EC152F157C11B
:104D500059F158C15AF178EC16F000C13BF501C188
:104D60003CF502C13DF503C13EF505015D67C0EFAD
:104D700026F05E67C0EF26F05F67C0EF26F0606741
:104D8000C4EF26F0D1EF26F05DC504F15EC505F154
:104D90005FC506F160C507F108EC20F003BF42EFE4
:104DA00027F059C13FF55AC140F5B5C541F5B6C523
:104DB00042F507940501110E326F899A400EC76EB5
:104DC000200EC66E9E96C69E060EC96EFF0E9EB63D
:104DD00002D0E82EFCD7898A899A9E96C69E020E3A
:104DE000C96EFF0E9EB602D0E82EFCD79E96C69ED8
:104DF00027C5C9FFFF0E9EB602D0E82EFCD79E96AF
:104E0000C69E26C5C9FFFF0E9EB602D0E82EFCD76F
:104E10009E96C69E25C5C9FFFF0E9EB602D0E82EFF
:104E2000FCD725EE33F0322F02D022EF27F09E96EA
:104E3000C69EDECFC9FFFF0E9EB602D0E82EFCD77D
:104E400013EF27F0898A899A9E96C69E050EC96E31
:104E5000FF0E9EB602D0E82EFCD79E96C69EC95283
:104E6000FF0E9EB602D0E82EFCD7C9B02DEF27F07A
:104E7000898A0501100E2527E86A2623E86A272378
:104E8000E86A2823120021C500F122C501F123C5DB
:104E900002F124C503F1899A400EC76E200EC66E3A
:104EA0009E96C69E0B0EC96EFF0E9EB602D0E82ED1
:104EB000FCD79E96C69E02C1C9FFFF0E9EB602D0C9
:104EC000E82EFCD79E96C69E01C1C9FFFF0E9EB676
:104ED00002D0E82EFCD79E96C69E00C1C9FFFF0EE9
:104EE0009EB602D0E82EFCD79E96C69EC952FF0EF3
:104EF0009EB602D0E82EFCD725EE33F00501100E49
:104F0000326F9E96C69EC952FF0E9EB602D0E82E04
:104F1000FCD7C9CFDEFF322F81EF27F0898A12003C
:104F2000899A400EC76E200EC66E9E96C69E900E43
:104F3000C96EFF0E9EB602D0E82EFCD79E96C69E86
:104F4000000EC96EFF0E9EB602D0E82EFCD79E96CC
:104F5000C69E000EC96EFF0E9EB602D0E82EFCD78C
:104F60009E96C69E000EC96EFF0E9EB602D0E82E1B
:104F7000FCD79E96C69EC952FF0E9EB602D0E82E62
:104F8000FCD7C9CF2DF59E96C69EC952FF0E9EB680
:104F900002D0E82EFCD7C9CF2EF5898A1200F4EC96
:104FA0001EF0B5C5E8FFD70802E3F4EC1EF0B5C566
:104FB000E8FFC80802E3F4EC1EF0B5C5E8FFB90845
:104FC00002E3F4EC1EF0B5C5E8FFAA0802E3F4EC36
:104FD0001EF0B5C5E8FF9B0802E3F4EC1EF02DECD3
:104FE00022F024EC26F0F29CF29E8B94C69AC2909A
:104FF0009482948C720ED36ED3A4FED789968A9035
:105000009390FF0EE8CF00F0E82EFED7002EFCD7DD
:105010008150F294F29A9E909D909E929D92F29869
:0C502000F292F290F286F28E0300FF0084
:10BF0000E844F926000C160C2B0C3F0C520C640C68
:10BF1000760C860C960CA50CB30CC10CCF0CDC0C6B
:06BF2000E80CF40C000C1B
:00000001FF
